S027000062696E2F64656D6F70726F675F6E75636C656F5F73746D33326631303372622E737265636D
S315080020000050002079220008C9220008C9220008C9
S31508002010C9220008C9220008C922000800000000D9
S31508002020000000000000000000000000C9220008AF
S31508002030C922000800000000C9220008812F0008F4
S31508002040C9220008C9220008C9220008C9220008B6
S31508002050C9220008C9220008C9220008C9220008A6
S31508002060C9220008C9220008C9220008C922000896
S31508002070C9220008C9220008C9220008C922000886
S31508002080C9220008C9220008C9220008C922000876
S31508002090C9220008C9220008C9220008C922000866
S315080020A0C9220008C9220008C9220008C922000856
S315080020B0C9220008C9220008C9220008C922000846
S315080020C0C9220008C9220008C9220008C922000836
S315080020D0C9220008C9220008C9220008C922000826
S315080020E0C9220008C9220008C92200080000000009
S315080020F000000000000000000000000000000000D2
S3150800210000000000000000005FF808F1EE11AA5573
S3150800211010B5054C237833B9044B13B10448AFF313
S3150800212000800123237010BD380400200000000041
S315080021308C32000808B5034B1BB103490348AFF3BB
S31508002140008008BD000000003C0400208C32000816
S3150800215070B50D4E0D4D761BB61006D00024013411
S3150800216055F8043B9847A642F9D1094E094D01F0A6
S315080021708DF8761BB61006D00024013455F8043BBA
S315080021809847A642F9D170BDD4320008D432000867
S31508002190DC320008D4320008024B13B1024800F0C2
S315080021A005B8704700000000B92100080023014661
S315080021B01A46184600F01EB838B50A4C0A4D641B74
S315080021C0A4100AD004F18043013B05EB8305013CCA
S315080021D055F804399847002CF9D1BDE8384001F084
S315080021E05BB800BFE0320008DC320008704700BF69
S315080021F0704700BF2DE9F0411D4C05462068904602
S315080022001F460E46FFF7F2FF1A4B1A68D2F84831F6
S315080022101BB35A6820681F2A24DC4DB9511C0232A8
S31508002220596043F82260FFF7E3FF0020BDE8F0811C
S31508002230012403EB820CCCF88880D3F888119440EB
S315080022402143022DC3F88811CCF80871E6D1D3F8DA
S315080022508C110C43C3F88C41E0E702F5A673C2F86B
S315080022604831D6E7FFF7C4FF4FF0FF30DEE700BF7F
S3150800227028040020B8320008DFF834D0002103E033
S315080022800C4B5B58435004310B480C4B42189A428E
S31508002290F6D30B4A02E0002342F8043B094B9A4264
S315080022A0F9D300F02DFEFFF753FF00F0DCFE704770
S315080022B000500020E032000800000020380400200A
S315080022C0380400200C050020FEE70000074AD36802
S315080022D023F4E0631B041B0C000200F4E0601843BF
S315080022E040F0BF6040F40030D060704700ED00E079
S315080022F030B4174BDB68C3F30223C3F10704042C7D
S3150800230028BF04241D1D062D01D9033B00E0002328
S315080023104FF0FF3505FA04F421EA0401994005FA5D
S3150800232003F322EA03031943002809DB0901C9B2AA
S3150800233000F1604000F5614080F8001330BC70473A
S3150800234000F00F000901C9B2024B1954F6E700BFA5
S3150800235000ED00E014ED00E00138B0F1807F0AD20C
S31508002360064B5860064AF02182F823100020986030
S3150800237007221A6070470120704700BF10E000E08E
S3150800238000ED00E0042805D0054A136823F004038D
S3150800239013607047024A136843F0040313607047DA
S315080023A010E000E0704708B5FFF7FCFF08BD000025
S315080023B0F0B482B000263546A0E0002A58D0012A9B
S315080023C010D1CE680EE06A4FBA4251D048D9694F4B
S315080023D0BA424DD007F58037BA4249D0A7F58017DB
S315080023E0BA4245D0FF2B57D88446FF2B57D8AC00A6
S315080023F0DCF800200F27A74022EA070206FA04F4B1
S315080024002243CCF800204A6812F0805F75D05A4AF9
S31508002410946944F001049461926902F00102019200
S31508002420019AAC08A71C554A52F8272005F003075D
S31508002430BF004FF00F0C0CFA07FC22EA0C0C504AAE
S31508002440904232D002F58062904271D002F58062E5
S3150800245090426FD002F58062904224D0042225E093
S31508002460A7F58017BA4203D007F58037BA42B9D123
S315080024708A687AB1012A08D044610826B2E7CE688C
S315080024800836AFE7CE680C36ACE704610826A9E73C
S315080024900026A7E70426A5E700F1040CA5E7A5F1A1
S315080024A00804A400A4E7032200E00022BA4042EA96
S315080024B00C020234314F47F824204A6812F4803F50
S315080024C03AD0304C22681A4322604A6812F4003F18
S315080024D038D02C4C62681A4362604A6812F4801F2E
S315080024E036D0284CA2681A43A2604A6812F4001F24
S315080024F034D0244CE2681343E36001350B6833FAA1
S3150800250005F231D00124AC4023409C42F5D14A68FB
S31508002510122AB7D03FF657AF022AB0D07FF64DAF92
S31508002520032AB5D0112A7FF45DAFCE68043659E781
S315080025300122BBE70222B9E7124C226822EA03020B
S315080025402260C2E70F4C626822EA03026260C4E7AF
S315080025500C4CA26822EA0302A260C6E7094CE268AC
S3150800256022EA0303E360C8E702B0F0BC704700BF85
S315080025700000211000003110001002400000014048
S3150800258000080140000401400AB1016170470904CE
S315080025900161704738B504460268136923F440534D
S315080025A0C1680B43136183680269134342691A437E
S315080025B00168CB6823F4B05323F00C031343CB60B4
S315080025C00268536923F4407381690B4353610268B7
S315080025D0214B9A421FD000F073FC00EB800000EB01
S315080025E0800063689B00B0FBF3F01C4DA5FB00322E
S315080025F05109642202FB110213013233A5FB03239E
S315080026005B0903F0F00202EB011203F00F032168E5
S3150800261013448B6038BD00F063FC00EB800000EBD0
S31508002620800063689B00B0FBF3F00C4DA5FB0032FD
S315080026305109642202FB110213013233A5FB03235D
S315080026405B0903F0F00202EB011203F00F032168A5
S3150800265013448B60DEE700BF003801401F85EB514D
S315080026602DE9F04105460F4616469846069C2B6806
S315080026701B6837EA03030CBF01230023B3421DD1AD
S31508002680B4F1FF3FF3D02CB100F002F9A0EB08003B
S31508002690A042ECD92A68D36823F4D073D3602A6899
S315080026A0536923F001035361202385F8393085F8EF
S315080026B03A30002385F83830032000E00020BDE8D2
S315080026C0F081704758B310B5044690F839300BB30B
S315080026D0242384F839302268D36823F40053D3605E
S315080026E02046FFF757FF2268136923F490431361C6
S315080026F02268536923F02A0353612268D36843F496
S315080027000053D3600020E063202384F8393084F82E
S315080027103A3010BD80F83830FFF7D3FFD8E70120EC
S3150800272070472DE9F04182B01E4690F83A30DBB288
S31508002730202B5AD104460D469046002959D0002A26
S3150800274059D090F83830012B57D0012380F838300B
S315080027500023C363222380F83A3000F099F807462D
S31508002760A4F82C80A4F82E801DE000963B46002293
S3150800277020212046FFF774FF002840D1236933B98A
S3150800278023685B68C3F3080325F8023B0BE023685C
S315080027905B68DBB225F8013B05E023685B6803F05C
S315080027A07F0305F8013BE38D9BB2BBB1E38D013B8B
S315080027B09BB2E385A368B3F5805FD6D000963B4607
S315080027C0002220212046FFF74BFFD0B92369002BB2
S315080027D0E3D123685B6805F8013BE4E7202384F826
S315080027E03A30002084F8380000E0022002B0BDE844
S315080027F0F0810120FAE70120F8E70220F6E7032036
S31508002800F4E70320F2E7000010B504460E4B1878EB
S315080028104FF47A73B3FBF0F30C4A1068B0FBF3F08D
S31508002820FFF79AFD68B90F2C01D901200AE00022AA
S3150800283021464FF0FF30FFF75BFD054B1C6000207B
S3150800284000E0012010BD00BF2C0400203404002045
S315080028503004002008B5074A136843F010031360D4
S315080028600320FFF733FD0020FFF7CEFF00F006FC3C
S31508002870002008BD00200240034A1168034B1B785C
S315080028800B441360704700BF080500202C04002085
S31508002890014B1868704700BF0805002082B0084B36
S315080028A01B68084AA2FB03235B0A00FB03F001909E
S315080028B000BF019B5A1E0192002BF9D102B0704746
S315080028C034040020D34D6210002800F0F18170B561
S315080028D082B00446036813F0010F2CD0AA4B5B683C
S315080028E003F00C03042B1DD0A74B5B6803F00C0305
S315080028F0082B12D06368B3F5803F41D0002B55D121
S3150800290003F1804303F504331A6822F480321A600F
S315080029101A6822F480221A6037E09B4B5B6813F42E
S31508002920803FE7D0984B1B6813F4003F03D06368D9
S31508002930002B00F0BF81236813F0020F75D0924B6D
S315080029405B6813F00C0F5FD08F4B5B6803F00C03CA
S31508002950082B54D02369002B00F089808B4B012269
S315080029601A60FFF795FF0546874B1B6813F0020FA1
S3150800297074D1FFF78DFF401B0228F5D903209EE18D
S31508002980814A136843F480331360636843B3FFF7DF
S315080029907FFF05467C4B1B6813F4003FCBD1FFF73E
S315080029A077FF401B6428F5D9032088E1B3F5A02FEB
S315080029B009D0754B1A6822F480321A601A6822F414
S315080029C080221A60E1E703F18043A3F53C331A68D5
S315080029D042F480221A601A6842F480321A60D4E7F8
S315080029E0FFF756FF0546684B1B6813F4003FA2D055
S315080029F0FFF74EFF401B6428F5D903205FE1624BC1
S31508002A005B6813F4803FA5D15F4B1B6813F0020F78
S31508002A1003D02369012B40F04F815B4A136823F0EA
S31508002A20F803616943EAC1031360236813F0080FCA
S31508002A3032D0A369002B5BD0554B01221A60FFF7F1
S31508002A4027FF0546504B5B6A13F0020F21D1FFF7AB
S31508002A501FFF401B0228F5D9032030E14A4A1368B4
S31508002A6023F0F803616943EAC1031360DDE7474BC6
S31508002A7000221A60FFF70CFF0546434B1B6813F04C
S31508002A80020FD2D0FFF704FF401B0228F5D9032016
S31508002A9015E10120FFF702FF236813F0040F00F089
S31508002AA09780394BDB6913F0805F33D1364BDA698F
S31508002AB042F08052DA61DB6903F080530193019B8F
S31508002AC00125344B1B6813F4807F25D0E368012B5E
S31508002AD036D0002B4CD103F1804303F504331A6A30
S31508002AE022F001021A621A6A22F004021A622CE023
S31508002AF0274B00221A60FFF7CBFE0546224B5B6A7E
S31508002B0013F0020FC8D0FFF7C3FE401B0228F5D901
S31508002B100320D4E00025D4E71E4A136843F48073E3
S31508002B201360FFF7B5FE06461A4B1B6813F4807F41
S31508002B30CCD1FFF7ADFE801B6428F5D90320BEE093
S31508002B40114A136A43F001031362E36873B3FFF78C
S31508002B509FFE06460C4B1B6A13F0020F37D1FFF790
S31508002B6097FE801B41F288339842F3D90320A6E0EA
S31508002B70052B11D0044B1A6A22F001021A621A6A4E
S31508002B8022F004021A62E0E7001002400000424206
S31508002B9080044242007000404D4B1A6A42F004021B
S31508002BA01A621A6A42F001021A62CEE7FFF770FE4D
S31508002BB00646474B1B6A13F0020F08D0FFF768FE5C
S31508002BC0801B41F288339842F3D9032077E0E5B9B0
S31508002BD0E369002B72D03E4A526802F00C02082ABA
S31508002BE056D0022B17D03B4B00221A60FFF750FE37
S31508002BF00446374B1B6813F0007F47D0FFF748FEA3
S31508002C00001B0228F5D9032059E0314AD36923F07D
S31508002C108053D361DCE72F4B00221A60FFF738FE9A
S31508002C2005462B4B1B6813F0007F06D0FFF730FED6
S31508002C30401B0228F5D9032041E0236AB3F5803FFB
S31508002C401AD023494B6823F47413226A606A024334
S31508002C5013434B601F4B01221A60FFF719FE044607
S31508002C601B4B1B6813F0007F0ED1FFF711FE001BEC
S31508002C700228F5D9032022E0154A536823F40033C5
S31508002C80A1680B435360DCE7002018E0002016E03B
S31508002C90012B16D00E4B5B6803F48031226A9142F1
S31508002CA011D103F47013626A93420ED1002006E034
S31508002CB001207047012002E0012000E0002002B058
S31508002CC070BD0120FBE70120F9E70120F7E700BF07
S31508002CD0001002406000424210B487B0164C94E8D7
S31508002CE00F000DF1180C0CE90F00238AADF804301B
S31508002CF0124B5B6803F00C02082A03D0104807B091
S31508002D0010BC7047C3F38342624412F8102C13F4C4
S31508002D10803F0CD0094B5B68C3F34043634413F808
S31508002D20143C074800FB02F0B0FBF3F0E7E7054860
S31508002D3000FB02F0E3E700BFA432000800100240DF
S31508002D4000127A0000093D00002800F0A08070B546
S31508002D500446534B1B6803F007038B420BD2504AB9
S31508002D60136823F007030B431360136803F0070384
S31508002D708B4240F08E80236813F0020F17D013F0B1
S31508002D80040F04D0474A536843F4E063536023684A
S31508002D9013F0080F04D0434A536843F46053536052
S31508002DA0404A536823F0F003A068034353600D4676
S31508002DB0236813F0010F31D06368012B20D0022B52
S31508002DC025D0384A126812F0020F64D035494A688D
S31508002DD022F0030213434B60FFF75AFD0646314BB8
S31508002DE05B6803F00C036268B3EB820F16D0FFF73B
S31508002DF04FFD801B41F288339842F0D9032045E005
S31508002E00284A126812F4003FE0D101203EE0254A24
S31508002E10126812F0007FD9D1012037E0204B1B68D9
S31508002E2003F00703AB420AD91D4A136823F00703C8
S31508002E302B431360136803F00703AB422DD12368B5
S31508002E4013F0040F06D0174A536823F4E063E168C9
S31508002E500B435360236813F0080F07D0114A5368D1
S31508002E6023F46053216943EAC1035360FFF734FF33
S31508002E700C4B5B68C3F303130B4AD35CD8400B4B6C
S31508002E8018600B4B1868FFF7BFFC002070BD0120C7
S31508002E9070470120FAE70120F8E70120F6E700BFAE
S31508002EA00020024000100240BC3200083404002012
S31508002EB030040020014B1868704700BF3404002016
S31508002EC008B5FFF7F7FF044B5B68C3F30223034A11
S31508002ED0D35CD84008BD00BF00100240CC320008C1
S31508002EE008B5FFF7E7FF044B5B68C3F3C223034A41
S31508002EF0D35CD84008BD00BF00100240CC320008A1
S31508002F000F4B1A6842F001021A6059680D4A0A40C6
S31508002F105A601A6822F0847222F480321A601A689B
S31508002F2022F480221A605A6822F4FE025A604FF48C
S31508002F301F029A60044B4FF000629A60704700BF08
S31508002F40001002400000FFF800ED00E008B5FFF7AA
S31508002F50B1FF084BA3FB00308009FFF7FDF90420F9
S31508002F60FFF710FA002211464FF0FF30FFF7C0F9BD
S31508002F7008BD00BFD34D621008B5FFF789FC08BD30
S31508002F8008B5FFF779FCFFF70EFA08BD08B5002269
S31508002F9020210248FFF7F8FA08BD00BF00080140E3
S31508002FA010B5FFF7E9FF0E4B1B68C31AB3F5FA7F96
S31508002FB00CD304460B4B1B784BB90122094B1A70EC
S31508002FC020210948FFF7E0FA054B1C6010BD0022D6
S31508002FD0044B1A7020210448FFF7D6FAF4E700BF1D
S31508002FE0580400205404002000080140014A024BFE
S31508002FF09A6070470020000800ED00E000B591B027
S31508003000012306934FF4A0220792002208920A93FE
S3150800301002230D934FF480330E934FF4E0130F936E
S3150800302006A8FFF751FC00B1FEE70F230193022122
S315080030300291002303934FF480620492059301A83A
S31508003040FFF782FE00B1FEE711B05DF804FB08B594
S31508003050FFF7CCFFFFF7FEFBFFF7D0FFFFF776FF82
S31508003060FFF794FF08BD08B5FFF7F1FF00F0A8F8D1
S31508003070FFF796FF00F006F9FAE70000F0B589B009
S315080030803B4B9A6942F001029A619A6902F0010281
S315080030900092009ADA6942F08052DA61DA6902F03F
S315080030A080520192019A9A6942F004029A619A69D9
S315080030B002F004020292029ADA6942F40032DA61F4
S315080030C0DB6903F400330393039B0320FFF7FEF841
S315080030D0002211466FF00B00FFF70AF9002211468D
S315080030E06FF00A00FFF704F9002211466FF0090095
S315080030F0FFF7FEF8002211466FF00400FFF7F8F814
S31508003100002211466FF00300FFF7F2F8002211467D
S315080031106FF00100FFF7ECF8002211464FF0FF3080
S31508003120FFF7E6F82027049701230593002506955F
S31508003130022607960F4C04A92046FFF739F92A46B6
S3150800314039462046FFF720FA0423049305960323FD
S31508003150079304A92046FFF72BF90823049305953E
S31508003160069504A92046FFF723F909B0F0BD00BF6C
S31508003170001002400008014008B50848084B0360E3
S315080031804FF46143436000238360C3600361836136
S315080031900C224261C361FFF795FA08BD5C04002062
S315080031A00044004008B50023012201460348FFF702
S315080031B0B8FA08B1002008BD0120FCE75C0400202D
S315080031C008B5FFF7D9FF08BDBFF34F8F0549CA6891
S315080031D002F4E062044B1343CB60BFF34F8F00BF8A
S315080031E0FDE700BF00ED00E00400FA0508B5214B35
S315080031F01B78B3B92048FFF7D5FF012800D008BDD2
S315080032001D4B1B78013BDBB23F2BF8D8FFF7B4FE0A
S315080032101A4B1860174B01221A70194B00221A70A4
S31508003220EDE7174B1B78013313481844FFF7BAFF2D
S31508003230012813D1124A13780133DBB213700E4AF0
S3150800324012789342DBD10B4A002111700A4A527850
S31508003250FF2AD4D1022BD2D1FFF7B6FFFFF78CFE97
S31508003260064B1B6864339842C9D9024B00221A7070
S31508003270C5E700BFDD0400209C040020E004002010
S31508003280DE04002008B5FFF7B1FF08BDF8B500BF9A
S31508003290F8BC08BC9E467047F8B500BFF8BC08BC29
S309080032A09E46704781
S315080032A402030405060708090A0B0C0D0E0F101075
S315080032B401020000000000200000000000000000D9
S315080032C401020304060708090000000001020304BA
S30D080032D49921000835210008C4
S309080032DC11210008A6
S315080032E000000000EC02002054030020BC0300206C
S315080032F000000000000000000000000000000000C0
S3150800330000000000000000000000000000000000AF
S31508003310000000000000000000000000000000009F
S31508003320000000000000000000000000000000008F
S31508003330000000000000000000000000000000007F
S31508003340000000000000000000000000000000006F
S31508003350000000000000000000000000000000005F
S31508003360000000000000000000000000000000004F
S31508003370000000000000000000000000000000003F
S31508003380000000000000000001000000000000002E
S315080033900E33CDAB34126DE6ECDE05000B000000F3
S315080033A0000000000000000000000000000000000F
S315080033B000000000000000000000000000000000FF
S315080033C000000000000000000000000000000000EF
S315080033D000000000000000000000000000000000DF
S315080037000000000000000000E404002001000000A2
S30D08003710100000000024F4007B
S7050800227957
